:100000000C9417020C94101B0C9434020C943402C0
:100010000C9434020C9434020C9434020C94340288
:100020000C9434020C9434020C9458220C942C231B
:100030000C94331D0C9434020C9434020C9434024E
:100040000C9434020C9434020C9434020C94340258
:100050000C9434020C94D61D0C9434020C9434028B
:100060000C9434020C9434020C9434020C94340238
:100070000C9434020C9434020C9434020C94340228
:100080000C9434020C9434020C9434020C94340218
:100090000C9434020C9434020C9434020C94340208
:1000A0000C9434020C9434020C9434022B0014008F
:1000B0001A000800150017002900040016000700A8
:1000C00009000A00E1001D001B00060019000500E0
:1000D0000551E000E200E30003512C002A00130068
:1000E00012000C0018001C00340033000F000E003A
:1000F0000D000B00280038003700360010001100FA
:100100004F0052005100500004512C002B001400ED
:100110001A00090013000A00290004001500160047
:1001200017000700E1001D001B0006001900050074
:100130000551E000E200E30003512C002A003300E7
:100140001C0018000F000D00340012000C00080005
:1001500011000B00280038003700360010000E0098
:100160004F0052005100500004512C002B0034006D
:100170003600370013001C0029000400120008009C
:1001800018000C00E100330014000D000E001B00ED
:100190000551E000E200E30003512C002A000F00AB
:1001A000150006000A0009003800160011001700AB
:1001B0000B00070028001D0019001A0010000500A0
:1001C0004F0052005100500004512C0035021E0215
:1001D0001F022002210222024C003A003B003C0098
:1001E0003D003E0001004000410042004300440049
:1001F0000100010001000100010001004C00270284
:100200002602250224022302310230022F022E028E
:100210002D023F000100010001006402320245008E
:10022000AE00A900AA00AB000100010035001E00CD
:100230001F002000210022004C003A003B003C003F
:100240003D003E00010040004100420043004400E8
:100250000100010001000100010001004C00270025
:100260002600250024002300310030002F002E003E
:100270002D003F0001000100010064003200450034
:10028000AE00A900AA00AB00010001000100005C63
:1002900001000100010001000100010001001D5CDE
:1002A0001E5C135C0100010001000100010001005F
:1002B0000100010001000100010001004C000100EB
:1002C000010001000100010001000100B45DB35D07
:1002D000B25D0A5C010001000100010001000100A3
:1002E0000100010001000100010001001C034C009D
:1002F0006500740073002000530070006C006900FA
:1003000074002000760032000000160357006F00D2
:100310006F0074007000610074006F006F00740063
:1003200000000403090409023B00020100A0FA09CD
:100330000400000103010100092111010001224014
:100340000007058103080001090401000103000002
:1003500000092111010001227B0007058203200012
:10036000011201000200000008776F020002000184
:1003700002000105010902A10185020901A1000590
:100380000919012908150025019508750181020543
:1003900001093009311581257F950275088106090B
:1003A000381581257F950175088106050C0A3802EC
:1003B0001581257F950175088106C0C0050109805A
:1003C000A101850319012AB700150126B70095017F
:1003D00075108100C0050C0901A101850419012ACD
:1003E000A002150126A002950175108100C005012B
:1003F0000906A101050719E029E71500250195085F
:10040000750181029501750881010507190029FF11
:10041000150026FF009506750881000508190129B9
:1004200005950575019102950175039101C011248F
:100430001FBECFEFDAE0DEBFCDBF11E0A0E0B1E03C
:10044000E4E7FBE402C005900D92AE39B107D9F79D
:1004500022E0AEE9B1E001C01D92A639B207E1F792
:100460000E942F140C94A2250C94000025E044E077
:1004700063E00E94BB020895FB01833B2DE59207D8
:1004800079F0843B2DE5920781F0823B9D4591F404
:100490008281882381F080E00E94A90280E0089593
:1004A0008281882341F081E0F7CF8281882319F08F
:1004B00082E0F2CF81E0089581E008950E943C023D
:1004C000089508950E9461020895A5E0B0E0EBE66A
:1004D000F2E00C940E2549835A833091A50189815D
:1004E0009A81311119C0662399F0222389F00E9464
:1004F0009108182F682F89819A810E946D0869815F
:100500007A81812F0E940B0F2596E3E00C942A2517
:100510000E947F08182FF3CF0E94910869817A8189
:10052000F1CFFC01262F408151816281738184814A
:100530000E946502089581E00895CF93DF93EC0156
:1005400060E00E949102BE010E946202DF91CF91A1
:100550000895CF93DF93C1E0D0E002C0CC0FDD1F40
:100560008A95E2F78C2F0E94B00CCE010E94900772
:10057000DF91CF910895E1E0F0E0DF0102C0AA0F22
:10058000BB1F6A95E2F7BD01DF0102C0AA0FBB1FC6
:100590004A95E2F7AD01462B572B02C0EE0FFF1F25
:1005A0002A95E2F79A01282339232417350719F4ED
:1005B0008E2B9F2B0895E095F0958E239F23089511
:1005C0000E94721008950E947610089508950E9466
:1005D0003B070E94E6022FEF84E39CE0215080401D
:1005E0009040E1F700C0000008950E94E7020E94D9
:1005F000FA1D08950E94E7020E940B1E08950F93B2
:100600001F93CF93DF938C0161E00E949102EC0174
:10061000B8010E945E02811106C080E0DF91CF9197
:100620001F910F910895B801CE010E94201A8823CE
:10063000A1F3B801CE010E94D816882371F3B80146
:10064000CE010E949219882341F3F8018281882308
:1006500061F0CB35FDE5DF0701F158F4C115ECE59C
:10066000DE0791F0CF3DDC4591F0C8010E945C02AD
:10067000D5CFCD358DE5D80769F090F0C83ADD4586
:10068000A1F70E94FA02C9CF0E94F502C6CF0E94CC
:100690004A0DF7CF0E94890CE8CF0E94930CE5CF5A
:1006A0000E94970CE2CF0E94101D0E9470030895D3
:1006B0000E9474030E94151D089508950E945D0311
:1006C000089581E008950E94610308950895CF93ED
:1006D000C82F0E945E038C2F0E946303CF91089560
:1006E00080E00E94670308950E94361C0E94670301
:1006F0000895CF930E94361CC82F8091A0018C17BB
:1007000079F0C093A0010E949F1D6093A101709396
:10071000A2018093A3019093A4018C2F0E946703F0
:10072000CF910895ABE0B0E0E8E9F3E00C940F2539
:100730004F83588769877A878B8761110E94D40B12
:100740001E821D8285E0FE013796DE011196019022
:100750000D928A95E1F78C819D81892B61F4498105
:100760005A816B817C818D819E810E94FD0A2B962E
:10077000E2E00C942B2589819A8189238F3F79F3BC
:10078000CE0101960E949B028111E9CFF0CFFC01BE
:10079000808191810E94C3080895CF93C82F882338
:1007A000C9F08238C9F40E94361C81FD13C089E368
:1007B0000E948C0B0E94F50B2FEF87EE93E02150E7
:1007C00080409040E1F700C0000089E30E94940B54
:1007D0000E94F50BCF9108958338A1F40E94361C36
:1007E00080FDF8CF83E50E948C0B0E94F50B2FEF64
:1007F00081EE94E0215080409040E1F700C000007D
:1008000083E5E4CF8438A1F40E94361C82FDE2CF58
:1008100087E40E948C0B0E94F50B2FEF81EE94E091
:10082000215080409040E1F700C0000087E4CECF27
:100830008CEF8C0F813AB8F48C2F0E94D71881115D
:10084000C9CF6C2F80910001909101010E94A11CE1
:10085000882329F08C2F0E94940B0E94F50B8C2F7B
:100860000E948C0BB5CF80E28C0F883048F4C770A3
:1008700081E001C0880FCA95EAF70E94B70BA8CFA4
:10088000EBE5EC0FE33040F4F0E0E25AFE4F8081FC
:1008900090E00E94631C9ECFE8E5EC0FE73150F436
:1008A000F0E0EE0FFF1FE05DFE4F808191810E941E
:1008B000791C90CFCD3E08F48DCF8C2F0E94B314BD
:1008C0000E94861587CF882309F455C0823879F4B1
:1008D0000E94361C81FF4FC089E30E948C0B0E944E
:1008E000F50B89E30E94940B0E94F50B0895833861
:1008F00059F40E94361C80FF3EC083E50E948C0B99
:100900000E94F50B83E5EECF843859F40E94361C23
:1009100082FF31C087E40E948C0B0E94F50B87E4B4
:10092000E1CF9CEF980F913AE8F290E2980F98305F
:1009300050F4877091E001C0990F8A95EAF7892FEA
:100940000E94BD0BD1CF9BE5980F933028F490E027
:1009500080E00E94631C089598E5980F973128F471
:1009600090E080E00E94791C08958D3E20F00E9466
:100970000D150E94861508951F93CF93DF93182FAE
:10098000EB010E94CD03209739F4812F0E9463046C
:10099000DF91CF911F9108958FE99FE00197F1F7C3
:1009A00000C000002197EFCF70E060E0893311F4C0
:1009B00060E570E00E94BC040895882321F00E9445
:1009C000B70B0E94F50B0895882321F00E94BD0B00
:1009D0000E94F50B0895B0E0A0E0E1EFF4E00C9484
:1009E00008256C01D62FC72FFC011281F580F294E7
:1009F0009FE0F9220E94AD0BE82E8823B9F0E12E8A
:100A00001123A1F08C2F807F803421F080E28D0FA4
:100A10008830D0F08091720282FF16C082E00E947E
:100A2000580C0E94AD0B91E0E82EE926BC2EB29442
:100A30008FE0B822FBE0FB1508F468C0EB2DF0E076
:100A4000EC55FA4D0C94F924E12CF0CF0C2F0F70DB
:100A5000C07F11F00295007F112399F0002359F017
:100A600080E28D0F883010F0D11107C0802F0E94D6
:100A7000B70B0E94F50B8D2F41C0802F0E94C70B32
:100A8000F8CF8D2F0E946304002309F43FC080E259
:100A90008D0F883010F0D11104C0802F0E94BD0B43
:100AA00003C0802F0E94CD0B0E94F50B2FC00C2F8E
:100AB0000F70C07FC03211F00295007FDD2381F0FE
:100AC000D13009F463C0112309F46DC0FF2009F48B
:100AD00063C0F601858180FFCECF8F7085835CC0B7
:100AE0008091720282FD33C0112359F0002329F056
:100AF000802F0E94B70B0E94F50B80E00E94CD036F
:100B000005C080E00E9463040111C7CFEB2DE850BF
:100B1000FF0B349720F40E94361C0E946703EE20DE
:100B200089F00E94A90B80FD0DC0F60112820E947F
:100B3000A30B0E94CB07C6010E94FB060E94A30BD9
:100B40000E94DB07CDB7DEB7E9E00C942425112322
:100B500089F0F11006C00E94D70B802B0E94DD04A3
:100B6000D5CF21E0F212F7CF0E94D70B802B0E9445
:100B7000DE0BCCCFF11006C00E94EB0B802F0E9441
:100B8000E404C4CF31E0F31609F2F6CF112331F0BB
:100B900085E08F1508F4BACF802FE0CF94E09F1541
:100BA00008F4B4CFEBCFFF2049F3D93349F4FFEF7A
:100BB00027EE33E0F15020403040E1F700C0000064
:100BC0008D2F0E946304A2CF8C2F8695869583700B
:100BD00069F0813009F09ACF8D2F9C2F93701111FD
:100BE00002C090E080E00E94791C90CF8D2F9C2F56
:100BF0009370111102C090E080E00E94631C86CFC8
:100C00008D2F112329F00E94B3140E9486157ECFE8
:100C10000E940D15FACF8C2F8370A1F5111176CF9C
:100C20004D2F429546954770440F440F2D2F2F703E
:100C300030E0042E02C0220F331F0A94E2F790E046
:100C400080E0D4FF09C08FE090E002C0880F991FB8
:100C50004A95E2F780959095C695C695C370822B0C
:100C6000932BC23049F058F4C13019F00E949C0710
:100C70004DCF0E9493074ACF0E94A50747CF0E94FD
:100C8000900744CF8695112311F08C2F8170882313
:100C900009F43CCF4D2F429546954770440F440FC1
:100CA0002D2F2F7030E0042E02C0220F331F0A9424
:100CB000E2F790E080E0D4FF09C08FE090E002C04E
:100CC000880F991F4A95E2F780959095C695C6952D
:100CD000C370822B932BC23049F058F4C13019F005
:100CE0000E94060813CF0E94FD0710CF0E940F0834
:100CF0000DCF0E94B1070ACFCF70112329F08C2F9E
:100D00000E94CB078D2F2ACF8D2F0E94E4048C2FB9
:100D10000E94DB07FBCED23F51F160F4D03FB9F027
:100D2000D13F81F0112309F449C0F110A4CE8C2FDA
:100D30008F7121C0D33F11F1D43FA1F7809172028E
:100D400082FD26C08C2F8F71112311F314C0112343
:100D500049F084E08F1508F4D9CE8C2F8F710E9452
:100D6000ED07D4CE95E09F1508F4D0CEF6CF8C2FAA
:100D70008F711111CDCF0E94CB07C8CE112329F05E
:100D80008C2F8F710E94BF07C1CE0E94BA07BECEC2
:100D9000112349F0CF718C2F0E94CB0763E08C2F79
:100DA0000E943A0CB3CE81E00E94580CE1E0EF15AE
:100DB00008F0ACCE82E00E94580CA8CEF110F5CE1F
:100DC0008C2F8F71A5CF0F931F93CF93DF93EC01DF
:100DD000688179818A810E94CE088C010E9418085E
:100DE0000E948F07B801CE010E94EB04DF91CF91E2
:100DF0001F910F910895CF93DF93EC018B819C811C
:100E0000892B29F08881998189238F3F51F4DF91C3
:100E1000CF910895CE010E94E306CE010E949D026B
:100E2000F6CFCE010E94FF028111F4CF0E94AD0BDC
:100E3000882369F38A81882351F38091720282FFAB
:100E4000E6CF82E00E94580CE2CF90E080E00E9462
:100E5000631C90E080E00E94791C0E94D40B0E94E9
:100E6000F50B0E94A2150E94861508950E949C0B06
:100E70000E94250708950E94C40B0E94360708951A
:100E800092959F70963091F058F4925F9F709230D7
:100E900058F4803F19F030F4883E30F481E0089532
:100EA0009A5FF4CF843FD1F380E00895883EB0F399
:100EB000813FD1F7F3CFFC0183819481892B29F005
:100EC0008081918189238F3F11F480E00895808192
:100ED00091810E94C3080E9440070895A5E0B0E0F8
:100EE000E4E7F7E00C940F252596E2E00C942B251F
:100EF000A6E0B0E0EEE7F7E00C940F252696E2E0DE
:100F00000C942B2508950E94820708950E94830760
:100F10009093C1018093C0010E9425070895089510
:100F20000E94860708952091C0013091C101822B53
:100F3000932B0E94860708952091C0013091C10132
:100F4000822393230E94860708952091C001309147
:100F5000C101822793270E94860708950E943602C6
:100F600008950E94AE079093BF018093BE010E9436
:100F70002507089590E080E00E94B107089521E0E0
:100F800030E0A90102C0440F551F8A95E2F7CA015B
:100F90000E94B107089521E030E002C0220F331F04
:100FA0008A95E2F78091BE019091BF01822B932B2D
:100FB0000E94B107089521E030E002C0220F331FE4
:100FC0008A95E2F7209530958091BE019091BF01FE
:100FD000822393230E94B107089521E030E002C0EC
:100FE000220F331F8A95E2F78091BE019091BF01D5
:100FF000822793270E94B10708952091BE01309166
:10100000BF01822B932B0E94B10708952091BE014E
:101010003091BF01822393230E94B107089520914C
:10102000BE013091BF01822793270E94B107089526
:101030000895262F277091E001C0990F2A95EAF7AD
:1010400023E0769567952A95E1F7660F771F660F7F
:10105000771FFA01E60FF71F50E040E0682F70E0BD
:101060008191DF0111979B01042E02C036952795CF
:101070000A94E2F7217021952827292328272C9309
:101080004F5F5F4F4430510559F70895A82FA7705F
:1010900023E0969587952A95E1F7880F991F880F89
:1010A000991FFB01E80FF91F50E040E080E021911B
:1010B00030E00A2E02C0369527950A94E2F7217097
:1010C0003327042E01C0220F0A94EAF7822B4F5FC8
:1010D0005F4F4430510559F70895262F983070F42A
:1010E000863060F4682F70E086E0989F600D711D77
:1010F000112446EA51E0822F0E9419080895292FF1
:10110000983068F4863058F490E066EA71E036E092
:10111000239F800D911D11240E944608089580E0B0
:101120000895B0E0A0E0E7E9F8E00C9408257C0120
:101130000091BE011091BF018091C0019091C10149
:10114000082B192BCFE0D0E0CC24C394D12CBC2E9B
:10115000C6010C2E02C0880F991F0A94E2F7802363
:101160009123892B49F4219790F7B12C8B2DCDB782
:10117000DEB7E9E00C942425B7018C2F0E94260FDE
:10118000019789F3F3CFCF93DF93EC010E9491088D
:10119000BE010E94260FDF91CF9108951F93CF9338
:1011A000DF93EB019091A501992339F0CB010E94C7
:1011B000C308DF91CF911F910895882369F0CB0177
:1011C0000E949108182F682FCE010E946D08BE0161
:1011D000812F0E94260FEDCFCB010E947F08182F90
:1011E000F6CF1F93CF93DF93C091C20116E0809199
:1011F000C3018C1304C0DF91CF911F910895D0E0FB
:101200001C9FF0011D9FF00D1124EC53FE4F4081F7
:10121000518162817381848195810E947807219632
:10122000C770E5CF4091F4015091F5016091F6014E
:101230007091F7018091F8019091F9010E9478076F
:1012400008951F93CF93DF938091F901807F09F078
:1012500049C08091F601882309F444C08091C201FD
:10126000C091C3016091F4017091F501A091F70163
:10127000B091F801D62FD72316E0C81799F190E066
:10128000109711F0DF3F19F401968770F6CF189F81
:101290009001199F300D1124F901EC53FE4F41814B
:1012A0004713F2CF40814613EFCF42814111ECCF7B
:1012B000438154814A1B5B0B483C510528F78091C0
:1012C000F9018F7080618093F901F901E753FE4FB6
:1012D00080818F708061808384EF91E00E94FB06A3
:1012E0000E94F108DF91CF911F910895A1E1B0E034
:1012F000ECE7F9E00C9407258C0185E0F801DE01AC
:101300001D9601900D928A95E1F7F801E28084EF35
:10131000C82E81E0D82E6091F7017091F801611517
:10132000710509F44EC19091F4012091F501892FC6
:1013300082238F3F09F445C140815181A380B4804D
:10134000F090F601F501E61BF70BFF2009F4EAC067
:101350008091F901382F307FE83CF10508F0A3C0F7
:1013600031116DC0FE2C251316C0941314C0E1106A
:1013700012C08F7080618093F9010E941209C6012A
:101380000E94FB068091F901F80185838F2D6196FB
:10139000EAE00C942325A114B10429F0842F8523BD
:1013A0008F3F09F027C180E0F82FF170DF2E80FF1A
:1013B0003CC08091C2012091C30136E0821315C068
:1013C0004D875E878D859E850E94C308292F2295B3
:1013D0002F702230F0F0243018F59F70F1F0F801F2
:1013E0009581907FD1F4D12C1EC090E0389FF00100
:1013F000399FF00D1124EC53FE4F6181651306C037
:101400006081641303C06281E6120FC00196877089
:10141000D5CF9F7011F0882331F3805E883018F3A8
:10142000C8010E94FB06FD2CB1CFEE2009F4AECF1F
:101430008091F90181608093F901F12CA7CF2513E8
:1014400006C0941304C0F801EE2009F487C0C80157
:101450000E945B07882319F1EE2009F18091F901C0
:10146000803270F02091F4013091F50138872F839C
:101470001986BB86AA868C87CE0107960E94FB063A
:1014800086E0F801A4EFB1E001900D928A95E1F7B2
:101490000E9421090E941209FF24F39477CFC8010A
:1014A0000E94FB06F9CF311113C07A2DB98AA88AA0
:1014B0006E2D89890E946E0784EF91E00E94FB06E1
:1014C00086E0F60111928A95E9F70E941209B5CFDC
:1014D00025130FC094130DC0E1100BC0F8018583D4
:1014E000C8010E94FB0686E0F60111928A95E9F791
:1014F0004DCFC8010E945B07882389F2EE2079F264
:101500008091F901803208F4BBCF2091F401309131
:10151000F5013A8329831B82BD82AC828E83CE0182
:101520000196ACCFE83CF10508F03EC0FE2CEE2061
:1015300009F4B5CF25132AC0941328C08091F9016E
:1015400080FD1BC0982F907FC1F0F8018583903FEC
:1015500031F0982F907F905F8F70892B8583C80121
:101560000E94FB0686E0F801A4EFB1E001900D9225
:101570008A95E1F70E94120909CF86E0F801A4EFED
:10158000B1E001900D928A95E1F700CFC8010E9469
:101590005B07811175CF8091F90181608093F9011A
:1015A000C8010E94FB06F2CE7A2DB98AA88A6E2D58
:1015B00089890E946E0786E0F60111928A95E9F703
:1015C000D9CFEE2009F46BCFC8010E945B07F82E3B
:1015D000882309F464CF86E0F801A4EFB1E001901C
:1015E0000D928A95E1F784EF91E00E94C7030E9473
:1015F0002109C0CF81E08E25D7CEACE0B0E0E3E09A
:10160000FBE00C940E254F83588769877A878B8778
:101610009C87CE0107960E947609882369F08A8507
:101620009B85892B39F04F815885842F85238F3FE7
:1016300009F06BC016E05FC086E0FE013796DE0160
:10164000119601900D928A95E1F78A859B85892BE9
:1016500089F38F81988589238F3F61F32091C3019E
:1016600030E0C9010196877099274091C20148175F
:10167000190671F40E943B071092C3011092C20137
:1016800086E0E4EFF1E0DF011D928A95E9F7D2CF21
:1016900096E0929FD001939FB00D1124AC53BE4FA2
:1016A000FE01319601900D929A95E1F78093C30166
:1016B0000E94F108BFCF819FC00111248C539E4F1F
:1016C0000E9476098823E9F0E091C2011E9FF00193
:1016D0001124EC53FE4F40815181628173818481DA
:1016E00095810E9478078091C20190E001968770F1
:1016F00099278093C2018091C2019091C3018913FF
:10170000DACF2C96E3E00C942A2569857A858B85BF
:101710009C850E9478078ECF682F80910001909160
:1017200001010E94D71C0895682F809100019091BB
:1017300001010E94DA1C089580910001909101013D
:101740000E94DD1C089580910202859585958595FE
:101750000895809102028770089590910202977017
:1017600081E009F480E0089580910D020895909140
:101770000D02892B80930D020895809590910D02A2
:10178000982390930D02089510920D020895909160
:101790000C02892B80930C020895809590910C0285
:1017A000982390930C02089510920C020895809152
:1017B0000302089508950E94DA0B08959091720231
:1017C00092FF08C090910302981721F080930302C2
:1017D0000E94DB0B089580910302882329F0109268
:1017E000030280E00E94DB0B0895CF93DF93E0912A
:1017F0000001F091010180910D028083E0910001D0
:10180000F0910101808190910C02892B808390914D
:101810000302992381F0E0910001F09101018081A0
:10182000892B808380910001909101010E948F1C7F
:1018300081110E94EB0BC0910001D091010148E0A1
:1018400050E06AEF71E0CE010E944A25892B59F0E1
:1018500088E0FE01AAEFB1E001900D928A95E1F7D0
:10186000CE010E944A1CDF91CF91089508950E94F5
:10187000360C08959091720292FF11C098E0899FF2
:1018800090011124622B609302020E94CB07809189
:1018900002028595859585950E94370C08950E94D2
:1018A000CB0708951092020280E00E94370C089541
:1018B000909102028095892380930202282F27703D
:1018C00091F4282F082E000C330B9217130659F0B1
:1018D0009091720292FF07C08595859585950E942B
:1018E000DB070E94520C08959091720292FB22270E
:1018F00020F9281769F080FB92F990937202809189
:101900007102909172020E94C40C82E00E94580CF5
:1019100008958091720282FB882780F991E08927DF
:101920000E94740C089581E00E94740C089580E078
:101930000E94740C089590E080E00E94682521E0E8
:10194000883E9E4F09F020E0822F089582E090E0CB
:101950000E946025089583E090E00E94602508952C
:10196000682F83E090E00E946E250895CF9384E075
:1019700090E00E946025C82F82E290E00E946025DE
:10198000982F8C2FCF910895CF93C92F682F84E083
:1019900090E00E946E256C2F82E290E00E946E25FE
:1019A000CF910895AB01BC018FE090E00E948025AB
:1019B0000895AB01BC0183E190E00E948025089569
:1019C00060E070E0CB010E94D90C089560E070E007
:1019D000CB010E94D20C0E94E00C089568EE7EEFCD
:1019E00090E080E00E948C2560E082E090E00E9420
:1019F0006E2560E083E090E00E946E251092C101A8
:101A00001092C00160E084E090E00E946E2564E0E6
:101A100082E290E00E946E2560E085E090E00E9406
:101A20006E2560E086E090E00E946E256FEF87E013
:101A300090E00E946E2540E050E0BA0188E090E01E
:101A40000E94802560E08DE090E00E946E2540E0DD
:101A500050E0BA0188E190E00E94802560E087E1D3
:101A600090E00E946E2540E050E0BA018CE190E0E9
:101A70000E94802570E060E080E290E00E948C256A
:101A800040E050E0BA0188E190E00E9480250E9489
:101A9000E60C08950E94EE0C0895682F8EE090E009
:101AA0000E946E2508950E949F1D60931C027093F2
:101AB0001D0280931E0290931F0260931802709380
:101AC000190280931A0290931B02089508950895B5
:101AD0000E94670D089508950E946B0D089580E59A
:101AE00090E10E942C1C0E94660D0E94680D0895D2
:101AF0000E9423120895089508950E947B0D0E946C
:101B00007C0D08950E9453100E94660308950E9460
:101B10008A1D0E9410100E943E120E9484110E9491
:101B2000820D0E94C0160E9448120E946C0D0895FA
:101B3000AAE0B0E0EEE9FDE00C9407250E94A711B1
:101B400080E1A82E82E0B82E750110E0F701019126
:101B50007F01812F0E9479101F5F183009F440C067
:101B60000817A1F38091200281FD0E947F100E943E
:101B7000780DC82E10E0812F0E947910082FF501F2
:101B800081915F01081731F1D02ED826F12CEE2477
:101B9000E3948D2D8E21B1F0CC20A1F0FE821F8325
:101BA00091E0802F8E2109F490E098870E94931D88
:101BB0008160782F9A8789874E815F8168858A85C1
:101BC0000E949203F394EE0CF6E0FF12E2CFF501CF
:101BD000319700831F5F183071F60E94530D20C0AB
:101BE0000813C0CF0E94931D8C0180910E0290912A
:101BF0000F0208171907A1F08FEF89838A831B82D0
:101C00000E94931D8160782F9D838C8349815A8126
:101C10006B818D810E94920310930F0200930E023C
:101C20000E9423120E94C4150E9479032A96EAE0BA
:101C30000C942325CF93DF930E942B0FEC01811589
:101C400021E5920708F042C0811530E5930708F0BE
:101C50009FC0883E910530F5803E910508F094C004
:101C6000883A910588F4853A910508F086C081305C
:101C7000910509F489C0009709F486C0049708F01B
:101C800083C0D0E0C0E080C08F3B9105D0F7C85A38
:101C9000D0E0CC0FDD1FCF59DE4F0990D881C02D89
:101CA000D46472C0811540E2940750F4C11581E0FC
:101CB000D80708F069C0CD3ED10518F3D06564C0DF
:101CC00081159044F0F2DF70D06A5EC0811535E571
:101CD000930718F5811544E5940708F085C0C115F0
:101CE00083E5D80708F06CC0C11522E5D20708F4D7
:101CF00062C0CE018370992721E030E002C0220F3C
:101D0000331F8A95E2F7C695C69580E2C89FE00129
:101D10001124C22BD32BDC6837C0811539E593071A
:101D2000A8F4811548E5940708F063C0C11586E55D
:101D3000D80708F0A6CF8C2F0E94CD0FC82FD0E077
:101D4000DC2FCC27CC27DF71D0621EC081152AE59D
:101D5000920708F453C090568115904208F091CF35
:101D60008D2F8F710E94CD0F90E0982F88278827A4
:101D70009F719C012C2BE901E7CFC55AD0E0C157D8
:101D8000DE4FC881D0E0D064CE01DF91CF910895BD
:101D90008370992721E030E002C0220F331F8A951B
:101DA000E2F7C695C69540E2C49FE0011124C22B1C
:101DB000D32BDD68E9CFDC2FCC27C16FD06AE4CF0D
:101DC000CE018370992721E030E002C0220F331F3B
:101DD0008A95E2F7C695C69540E2C49FE0011124BA
:101DE000C22BD32BDA68D0CFD82FCC27C46FD06AC0
:101DF000CBCFD82FCC27C06FD06AC6CF8F700E94B0
:101E0000CD0F34E0D695C7953A95E1F7CF709C2F6A
:101E1000EC01D069B9CF972F7830A8F4663098F4E8
:101E200070E026E0929F600D711D1124FB0190E38C
:101E3000899FE00DF11D1124EE0FFF1FE455FF4FA8
:101E400085919491089580E090E008950E940B0F91
:101E50000E941A0E089582389105B9F1B0F48133C9
:101E6000910509F47DC048F48932910509F46DC0EB
:101E70008A32910509F47BC008958533910509F4F0
:101E80005FC08933910509F10895833E9105D9F129
:101E900038F4803E910529F1823E910579F108954B
:101EA000863E9105D9F1873E910509F43EC0843EF6
:101EB000910541F52091720221FF24C080917102A9
:101EC00084FD19C087EE90E008952091710223707F
:101ED00009F05AC02091720223FF14C089E290E0F9
:101EE00008952091710220FD38C03091720230FFB8
:101EF00009C024FF43C090E080E008952091710262
:101F000022FDF7CF08952091710222FD3AC0309151
:101F1000720230FD39C024FFF5CFEDCF2091710260
:101F200023FFF0CF24FDE7CFCDCF2091710223FD19
:101F30002EC03091720231FFEECF84EE90E0089512
:101F40002091710225FFDECFC9CF2091710225FDBE
:101F500021C02091720223FFD5CF89E390E0D2CF38
:101F60002091710226FFCECF8AE290E00895209161
:101F7000710226FFC7CF81E390E0089583EE90E0E1
:101F8000089582EE90E0089580EE90E0089586EE48
:101F900090E0089585E390E008959091710292FF9A
:101FA00006C0282F28712830F9F4877F846093FFBA
:101FB00006C0282F28712831F1F4877E8461209192
:101FC000720220FF06C0382F38713830D9F4877F6D
:101FD000816021FF06C0282F28712831D1F4877E27
:101FE000816194FD877E0895282F24712430F9F6AD
:101FF0008B7F8860DCCF282F2471243101F78B7E02
:102000008861DDCF382F3171313019F78E7F8860CC
:10201000E0CF282F2171213121F78E7E8861E1CF19
:1020200010926D0210926E0210926F021092700266
:102030000895CF92DF92EF92FF926B017C010E9494
:10204000231281110EC00E949F1DC61AD70AE80AEA
:10205000F90AC0926D02D0926E02E0926F02F09285
:102060007002FF90EF90DF90CF9008950F931F9331
:102070000E942312882329F00E949F1D1F910F9117
:1020800008950E949F1D00916D0210916E02209193
:102090006F0230917002600F711F821F931FEECF8D
:1020A00080E0089508950E949B0C811102C00E9457
:1020B0004A0D0E94A60C809320020E94B60C9093B9
:1020C0007202809371020E9452100E94AB0C90E049
:1020D0000E9490078091BE019091BF010E94AE07BF
:1020E000089508950E947110089508950E94751032
:1020F0000895E82FF0E0E458FD4F80810895089599
:1021000080EA8A95F1F7089500C008950E94801032
:10211000089508950E9489100895EF92FF921F93E9
:10212000CF93DF9300D000D0CDB7DEB70E9423124B
:10213000182F60918402882309F447C019821A82FB
:102140001B821C82862F90E09E012F5F3F4F7901FA
:10215000B90184589D4F0E9456128823E9F080915E
:10216000730290E044E050E0B70184589D4F0E9414
:102170004A2521E020932102892BC9F410E00E9416
:10218000E302812F0F900F900F900F90DF91CF916E
:102190001F91FF90EF90089580912102882371F3A1
:1021A00084E0F70111928A95E9F710922102E091FB
:1021B0007302F0E0E458FD4F89819A81AB81BC81C4
:1021C00080839183A283B383DACF70E064587D4F1C
:1021D0008091730290E084589D4F0E94DD120E940E
:1021E0008A10CFCFF894E82FE295EF70F0E031A19C
:1021F000282F2F7081E090E001C0880F2A95EAF720
:10220000982F9095932391A392A1892B82A37894E0
:102210000895CF93DF9387E90E94F21086EC0E9425
:10222000F21084E30E94F21085E30E94F210C2E9EA
:10223000D1E089918F3F11F00E94F21081E0C839FE
:10224000D807B9F7DF91CF910895B0E0A0E0EBE2B5
:10225000F1E10C940925EC01D62E062F10E0C801FF
:1022600088569E4F7C01FC0180818F3F09F445C058
:10227000F894E82FE295EF70F0E091A18F7021E0E3
:1022800030E001C0220F8A95EAF7892F822B81A3C3
:1022900082A12095282322A378940E948410E2E949
:1022A000F1E048E951E031E0C12C21912F3F51F19B
:1022B000A22FA295AF70B0E090968C9190E02F7015
:1022C00002C0959587952A95E2F780FD1BC0832F64
:1022D000C82A330F4E175F0741F7F70180818F3F00
:1022E00011F00E94F21061E0C11001C060E08D2D7C
:1022F0000E948610C00FD11FC882CDB7DEB7E8E0BC
:102300000C94252580E0E4CF8091020180910201A8
:1023100094E0811190E09093840284E0891B809383
:1023200073020E94091188E0ECE7F2E0DF01982FC8
:102330001D929A95E9F7E4E7F2E0DF011D928A9594
:10234000E9F784E00E94E5110E94E0020895A8E008
:10235000B0E0EDEAF1E10C940C258E010F5F1F4F08
:1023600088E0F80111928A95E9F7F12C6F2DC801E8
:102370000E942511F394F4E0FF12F8CF48E050E0FA
:10238000B80184E792E00E944A2521E0009709F411
:1023900020E0892B41F088E0F801A4E7B2E0019049
:1023A0000D928A95E1F76091840270E064587D4F48
:1023B00044E084E792E00E94E611182F0E948D10FD
:1023C000812B2896E5E00C9428250895CF92DF9282
:1023D000EF92FF920F931F93CF936C017B01042F19
:1023E000222349F081E0809324020E94931D909360
:1023F000230280932202C0912402C1110AC0C0E0CE
:102400008C2FCF911F910F91FF90EF90DF90CF9085
:10241000089580912202909123020E94AB1D05979E
:1024200070F310E0A801B601C7010E944A25892B6C
:1024300041F0A801B601C7010E945725109224025D
:10244000DFCFC0E0FBCF80912702811107C00E943F
:10245000D824882351F081E08093270281E0909175
:102460002702913009F080E0089582E080932702EE
:102470000E94D324F3CF0E94231208950E943B129E
:10248000809302010E94231281110E948C120895F0
:102490000E942312811102C00E948F12089581E0D0
:1024A000909128029A3008F080E008950F931F93CE
:1024B000CF93DF93EC018B01809128028A30B8F42E
:1024C000B801CE010E94DA12C82F811122C080917A
:1024D00028028F3FB9F40E94931D909326028093A7
:1024E00025028C2FDF91CF911F910F91089580913C
:1024F0002502909126020E94AB1D843F914000F777
:10250000C0E0EFCF8F5F809328028A3020F7C1E0D0
:10251000E8CF10922802E5CF0E94CA1A08950E94BF
:10252000CD1A0895B0E0A0E0E8E9F2E10C940A25A4
:102530007901C82F880FDD0B41155105A9F0FE0167
:1025400093E0EE0FFF1F9A95E1F7ED5FFE4F81815B
:102550009281875D9D4F208130E04217530708F438
:102560009A01A9010E945725CE010E94B61BD82EC0
:102570008823D1F001151105B9F083E0CC0FDD1FE0
:102580008A95E1F7FE01ED5FFE4F438150E00417AD
:10259000150708F4A801CD5FDE4F6C817D81675D72
:1025A0007D4FC7010E9457258D2DCDB7DEB7E7E0DF
:1025B0000C9426250E94D41308950E94EB130895CD
:1025C000A4E0B0E0E6EEF2E10C940D2560913E024D
:1025D00070913F0280914002909141020E94BA1D89
:1025E00011E0643671058105910518F10E943610DD
:1025F0006E5F7F4F8F4F9F4F69837A838B839C835E
:1026000010E000E030E020E044E050E0BE016F5F09
:102610007F4F82E00E949212182F882351F00E946F
:102620009F1D60933E0270933F02809340029093FF
:102630004102812F2496E4E00C942925B0E0A0E02B
:10264000E4E2F3E10C9407257C015B016A010E943E
:102650004F1201E010E0882311F00AE010E0C1E021
:10266000D0E0B501C701F6010995811104C021969A
:102670000C171D072CF4CDB7DEB7EAE00C94232528
:10268000CC9F9001CD9F300D300D112490E080E063
:1026900045E34A95F1F70000019682179307C1F7C9
:1026A000E0CFA5E0B0E0E7E5F3E10C9407255B019E
:1026B000E0909C01F0909D0101E010E09E012B5FF5
:1026C0003F4F50E040E070E060E080E00E949212F6
:1026D000182F882309F44BC067018FEFC81AD80A56
:1026E00060913A0270913B0280913C0290913D02D0
:1026F0000E94BA1D643671058105910580F104E0E0
:1027000010E09E012F5F3F4F50E040E070E060E03E
:1027100081E00E949212F82E64E070E0C6010E94EF
:10272000C11611E09D81981310E01F2159F10E94FC
:102730009F1D60933A0270933B0280933C029093FA
:102740003D0289819A81AB81BC818093360290934E
:102750003702A0933802B093390211E013C064E04D
:1027600070E0C6010E94C1169D818913C8CFF70190
:1027700081819281A381B48189839A83AB83BC8355
:102780001111DFCF8091360290913702A09138026B
:10279000B0913902F50180839183A283B383812FA5
:1027A0002596EAE00C9423250F931F93CF93DF9394
:1027B000EC018B0141E553E10E941E13882331F0A7
:1027C00040EE52E1B801CE010E941E13DF91CF917D
:1027D0001F910F9108950F931F93CF93DF93C09193
:1027E0009C01D0919D01CE01019624E0FB01DC010A
:1027F00001900D922A95E1F764E070E00E94C11605
:1028000088836D817E818F8198850091320210913D
:10281000330220913402309135026017710782072C
:10282000930751F060933202709333028093340225
:10283000909335020E941910DF91CF911F910F9153
:1028400008950E94AE1F0E94870D0E94BB1F08952D
:102850000E94C01F0E94980D0E94DA1F08950E94D6
:102860002C1D0E94941F0E946F0D0E9421140E9433
:1028700028140E947D0DFBCF8091480280FF0DC07F
:102880006091200170E0660F771F6038710570F568
:102890006115710569F1862F089581FF07C0609168
:1028A000200184E0689FB0011124EFCF60912001E6
:1028B00082FD0AC0809147028823A9F020911F0160
:1028C00060912001821710F088E0ECCF869FC00154
:1028D000112433E0880F991F3A95E1F7622F70E0D9
:1028E0000E94E524D2CF68E070E0D5CF8FE708954D
:1028F00081E008958091480280FF0CC060911C0126
:1029000070E075956795759567956115710549F145
:10291000862F089581FF06C060911C0170E07595B7
:102920006795F3CF60911C0182FD0BC09091460228
:102930009923A1F060911B0180911C01961738F03A
:10294000682F70E06038710500F38FE70895899F64
:10295000C001112470E00E94E524F4CF61E070E032
:10296000D7CF81E008958D3E31F40E943C148195CB
:1029700080934C0208958E3E19F40E943C14F8CFC7
:102980008F3E31F40E943C14819580934B02089550
:10299000803F19F40E943C14F8CF893F29F40E942B
:1029A0007A1480934D0208958A3F21F40E947A148C
:1029B0008195F7CF8B3F31F40E947A1481958093F3
:1029C0004E0208958C3F19F40E947A14F8CF9FE0CC
:1029D000980F983070F4815F990B21E030E001C0CE
:1029E000220F8A95EAF780914A02822B80934A024D
:1029F00008958D3F31F480914802816080934802B0
:102A000008958E3F21F4809148028260F7CF8F3F76
:102A1000B9F7809148028460F1CF40914B028D3E1E
:102A200059F480914C0287FF0DC010924C02411165
:102A30000BC01092470208C08E3E81F480914C0278
:102A400018169CF3442381F080914D0290914E0220
:102A5000892B09F05AC01092460208958F3E49F41E
:102A600047FFF0CF10924B0280914C028111ECCFC6
:102A7000E0CF803F19F41416ACF3E4CF90914D02EF
:102A8000893F29F41916F4F610924D02DBCF8A3FE4
:102A900019F497FFD7CFF8CF90914E028B3F29F4CE
:102AA00097FFD0CF10924E02CDCF8C3F19F419165C
:102AB000CCF3C8CF9FE0980F983090F4815F990BCA
:102AC00021E030E0B90102C0660F771F8A95E2F776
:102AD000CB01809590914A02892380934A02B2CF1C
:102AE0008D3F31F4809148028E7F80934802AACFB7
:102AF0008E3F21F4809148028D7FF7CF8F3F09F000
:102B0000A1CF809148028B7FF0CF08950E94931D42
:102B10009C0190914B0280914C02982B21F03093B4
:102B200045022093440290914D0280914E02982BD1
:102B300021F0309343022093420289E492E00E9404
:102B4000551C089586E0E9E4F2E0DF011D928A95C4
:102B5000E9F7109247021092460210924802089537
:102B6000FC01828181110EC0838181110BC084819F
:102B7000811108C091E08581811101C090E0892F09
:102B80008170089581E0FCCFA6E0B0E0EAECF5E1C9
:102B90000C940E2586E0E9E4F2E0DE011196019046
:102BA0000D928A95E1F710924B0210924C0210920E
:102BB0004D0210924E028B819C81892B89F080916D
:102BC0004402909145020E94AB1DAC0190914702D6
:102BD0009923C9F1809121018417150608F440C09A
:102BE0008D819E81892B91F08091420290914302C8
:102BF0000E94AB1DAC0190914602992309F471C06B
:102C000080911D018417150608F479C0BE016F5F1D
:102C10007F4F89E492E00E94E41C811105C089E4A1
:102C200092E00E94B01581110E94861586E0FE0197
:102C30003196A9E4B2E001900D928A95E1F72696CB
:102C4000E3E00C942A25209122018AE0289F90013C
:102C500011242417350720F69F5F9093470202C086
:102C60009F3FD1F71B81112359F00E943C149FEF25
:102C700011160CF491E0899F802D112480934B0252
:102C80001C81112359F00E943C149FEF11160CF483
:102C900091E0899F802D112480934C0230914B024A
:102CA000332309F49DCF20914C02222309F498CFBD
:102CB00045EB3403C0011124992359F090934B0242
:102CC00045EB240390011124332339F030934C0257
:102CD00087CF81E080934B02F3CF81E080934C0259
:102CE0007FCF20911E018AE0289F90011124241794
:102CF000350708F08BCF9F5F9093460202C09F3F3D
:102D0000D1F71D81112359F00E947A149FEF1116FB
:102D10000CF491E0899F802D112480934D021E8137
:102D2000112359F00E947A149FEF11160CF491E0D0
:102D3000899F802D112480934E0230914D023323C0
:102D400009F464CF20914E02222309F45FCF45EBB2
:102D50003403C0011124992359F090934D0245EB9F
:102D6000240390011124332339F030934E024ECFC7
:102D700081E080934D02F3CF81E080934E0246CFF5
:102D80000895FC01680F791F8FEF91E36E177F079D
:102D900009F408952191822728E030E087FF06C0DA
:102DA000880F892721503109C9F7F0CF880FFACF52
:102DB000CF93DF93EC01FB018281882309F464C186
:102DC000C430FDE5DF07E0F5CB3F9CE5D90730F4E3
:102DD0009E0122503C4524313105D8F50E94B60CA5
:102DE0009093720280937102C231ECE5DE0709F420
:102DF0001FC108F06EC0C9308CE5D80709F4F2C0D5
:102E000008F03FC0C530ECE5DE0709F4DBC058F53B
:102E1000C3308CE5D80709F4CDC008F0CFC080914D
:102E200071028160C230DC4509F4AEC0809171024C
:102E3000909172020E94C40C0E943B0780E009C07E
:102E4000C63AEDE5DE0751F238F4C2369DE5D90702
:102E500029F2DF91CF9108959E012E5A3D452330EE
:102E60003105B8F7BBCF809171028062C730FCE5B5
:102E7000DF0709F489C008F4B1C080917102806451
:102E800083C0CD309CE5D90709F4BAC070F48091B5
:102E900071028E7FCB30FCE5DF0709F475C008F4C2
:102EA000A7C0809171028D7F6FC0CF309CE5D9079C
:102EB00009F4B6C008F4A8C0C031FCE5DF0709F486
:102EC000B3C0C131DC4509F0B1CF809171028F7B75
:102ED0005BC0C1159DE5D90709F4B4C098F5CB3F97
:102EE000FCE5DF0709F472C0B8F4C4319CE5D907EA
:102EF00009F4B6C008F4A2C0C531DC4509F096CF8C
:102F00008091710282FB992790F921E0922790FB32
:102F100082F990FB83F938C0CD3F8CE5D80709F4DE
:102F200077C008F457C0CE3FECE5DE0709F474C063
:102F3000809172028360CF3FDC4509F077CF8093A8
:102F4000720274CFC2368DE5D80709F496C068F4D2
:102F5000C230EDE5DE0709F48CC008F477C0C33059
:102F6000DD4509F063CF80E085C0CE3A9DE5D90705
:102F7000E9F068F490917102892F8E7F90FF816053
:102F8000C63ADD4509F052CF809371024FCFCF3A58
:102F90008DE5D80789F1C03BDD4509F047CF909119
:102FA0007202892F877F93FF8860C9CF8091720258
:102FB0008860C5CF809171028260E6CF80917102F6
:102FC0008460E2CF809171028860DECF80917202CE
:102FD0008160B5CF809172028260B1CF8091710221
:102FE0008061D2CF0E943B07809171028068CCCF74
:102FF000809171028C60C8CF80917202877F9FCFD1
:10300000809171028B7FC0CF80917102877FBCCF8E
:10301000809172028E7F93CF809172028D7F8FCFCD
:10302000809171028F7EB0CF809171028F7DACCF85
:103030000E943B07809171028F77A6CF8091710229
:10304000837FA2CF809172028C7F79CF80917202B0
:10305000982F909591708E7F892B90FB81F96FCF7F
:103060000E943B0790917102892F97FB87F9805846
:103070008BCF81E00E944D0DD9CE90917102892FA6
:103080008F7E94FF806180CF81E0E3CE8B3109F4A5
:1030900065C040F58B3071F078F4863009F447C094
:1030A00020F4853059F180E00895873009F448C054
:1030B0008830C9F781E00895803109F45DC068F473
:1030C0008E3089F790912002892F8B7F92FF846048
:1030D0008093200282FD4CC0EDCF863159F38931B7
:1030E00049F3E1CF8A3201F160F48732B1F020F484
:1030F0008E31C8F28D514CC08932A9F60E94F5027A
:10310000D9CF833440F48A3308F041C0853329F0A5
:10311000883381F2C8CF833431F681E090E00E9499
:1031200090070E943B07C6CF0E944A0DC3CF8091F3
:103130002002807F8093200281E0809352020895D4
:1031400090912002892F8E7F90FF816080932002D2
:1031500080FDB0CF817F80932002ACCF9091200280
:10316000892F8D7F91FF82608093200281FFA2CF03
:10317000809120028160EFCF90912002892F877F7C
:1031800093FF88608093200283FDF2CF93CF895311
:1031900021E030E0A90102C0440F551F8A95E2F7F3
:1031A000CA01BDCF80E008950E94D2180895CF9340
:1031B000C82F809152028130B9F0882331F08230DB
:1031C000A1F11092520280E00DC00E94B40B823235
:1031D000D1F78C2F0E94D21881111BC08C2F0E9416
:1031E00046188170CF9108950E94B40B823289F302
:1031F0008C2F0E94D41881110AC0C43199F060F458
:10320000CB3029F0C03169F782E08093520281E02F
:10321000E8CF81E090E0E5CFC93221F0C833B9F3BF
:1032200080E0DFCF10925202FBCFC93209F440C0D8
:10323000F0F4C431E9F1A8F481E0C73099F6809345
:10324000220184E1809321018AE0809320018EE1B4
:1032500080931F0188E080931C0188E280931B010A
:1032600004C082EE8C0F8A3070F181E0BBCFC03594
:1032700009F450C0B8F48AE0CF34B9F7E0914F02B6
:10328000F0915002309789F32081082E000C990BA1
:10329000820F911D8F3F910509F00CF43FC08FEF15
:1032A0008083E3CFC135C1F181E0C23539F39ACFD4
:1032B000809151028823C9F210925102109250025B
:1032C00010924F02D2CFCD51C0935102C330C9F0FA
:1032D00048F4C13099F081E291E0C23051F010928F
:1032E0005102C3CFC53099F078F08BE191E0C63040
:1032F000B1F79093500280934F02B7CF82E291E0F2
:10330000F8CF80E291E0F5CF8FE191E0F2CF8CE150
:1033100091E0EFCF86EFB2CF8FEFB0CF97FFC0CF66
:103320001082A3CFCF93DF93EB0186319C4511F53B
:103330000E94B40B9A81992399F08A7A91E009F45A
:1033400090E090935302811109C089E20E948C0B96
:103350000E94F50B80E0DF91CF91089585E3F6CFD1
:1033600080915302811104C089E20E94940BF0CF36
:1033700085E3FBCF81E0EFCF0F931F93CF93DF93D4
:10338000C42FD22FFC0182818823C9F040935602BA
:103390000E94931D909355028093540280E28C0FFB
:1033A000883040F4C77081E001C0880FCA95EAF701
:1033B0000E94DD04DF91CF911F910F91089510912C
:1033C0005602141332C080915402909155020E940B
:1033D000AB1D883C910548F5C0E2CD0F1D17B9F033
:1033E00080E2810F883040F4177081E001C0880FBF
:1033F0001A95EAF70E94E404C83048F481E09D2F52
:10340000977001C0880F9A95EAF70E94DD04802F1B
:103410000E94D404C83070F6D77081E001C0880FD4
:10342000DA95EAF70E94E404C5CF80E28C0F883079
:1034300008F6C77081E001C0880FCA95EAF7F2CF9D
:103440000F939C01CB01243F4CE5340759F1A8F4BC
:10345000293DFCE53F0701F12A3D4CE53407D1F158
:10346000283D3C4591F406E221EE41EE68ED7CE515
:103470000E94BC1980E00F910895263FFCE53F07AC
:10348000E9F0B0F0273F3C45F9F0FC018281882348
:1034900039F110925602EFCF07E225EE45EE69EDC5
:1034A0007CE5E6CF06E221EE40EE64EF7CE5E0CF7E
:1034B00007E225EE44EE65EF7CE5DACF06E221EE89
:1034C00042EE66EF7CE5D4CF07E225EE46EE67EFED
:1034D0007CE5CECF08E221E045EE6AED7CE5C8CF81
:1034E00081E0C9CF8EE1489B02C08150E1F7489B43
:1034F000FECF0895589880E28A95F1F7589A08957A
:10350000FC013BE03A95F1F798E020E080E031E003
:1035100040E14A95F1F7880F489B02C0816023275C
:1035200042E04A95F1F7000040E14A95F1F79150E9
:1035300079F790E19A95F1F799B132E03A95F1F780
:10354000000040E14A95F1F7917092272081920F97
:1035500090830895A1E0B0E0E0EBFAE10C940B2534
:1035600019828C017C01E60EF11C0E151F0541F439
:1035700081E09981911180E02196E6E00C94272565
:103580000E94721ACE0101960E94801AF80181935E
:103590008F01EBCF509A589A08955098589AE89A0C
:1035A000E9E6F0E080818C7F808308956150770B9D
:1035B00091E001C0990F6A95EAF720E031E091119E
:1035C00008C0222391F0589A80E28A95F1F7589822
:1035D0000895492F482339F0589A232740E24A9505
:1035E000F1F79695ECCF5898F9CF5898EDCFFF9218
:1035F0000F931F93CF93DF93EC018C01060F111DE6
:10360000C017D10729F4CDB7DEB7E5E00C94282523
:10361000F9900E947A1A68E08F2D0E94D61AF0CF96
:103620001F920F920FB60F9211240F931F932F9397
:103630003F934F935F936F937F938F939F93AF933A
:10364000BF93EF93FF93CF93DF930F92CDB7DEB786
:1036500019820E94721ACE0101960E94801A082FC8
:10366000069506950695282F22952570902F957022
:10367000290F922F937026952695920F9827977071
:103680008981982B09F05CC0043008F059C080E1B2
:103690008A95F1F7589A509A82E08A95F1F700C01E
:1036A000589888E0089F80011124D801AD5FBE4F73
:1036B0001696ED91FC9117973097A9F060919C01B7
:1036C00070919D0114962D913C911597260F371FEF
:1036D00011968D919C911297680F791F13964C91BA
:1036E00013978C910995F801ED5FFE4F6381662376
:1036F00051F020919C0130919D0184819581820F30
:10370000931F0E94F71A0E947A1A80E18A95F1F7B6
:1037100058985098589A80E18A95F1F7F801ED5F32
:10372000FE4F6081662351F020919C0130919D01F4
:1037300081819281820F931F0E94AA1A0E94721A9D
:103740000F90DF91CF91FF91EF91BF91AF919F913A
:103750008F917F916F915F914F913F912F911F9129
:103760000F910F900FBE0F901F9018950F931F93FE
:10377000CF93DF93EC0104970CF04CC0F894509A6F
:10378000589885E08A95F1F700009C2F96959570E2
:103790008C2F8570980F892F83709695969523E0CE
:1037A000CC0FDD1F2A95E1F7980F8E01092B0E949F
:1037B0007A1A00C068E0802F0E94D61A80E18A95AC
:1037C000F1F75098589A489B1EC087E090E04899BE
:1037D0001CC0FE01ED5FFE4F63816623F9F020916E
:1037E0009C0130919D0184819581820F931F0E94DD
:1037F000AA1A811113C0509A589A7894DF91CF91E8
:103800001F910F91089500C0DECF019729F4509ABF
:10381000589A789480E0F2CF00C0D9CF0E94721AF3
:1038200080E28A95F1F75898509A80E18A95F1F7ED
:10383000CD5FDE4F6881662351F020919C0130916D
:103840009D0189819A81820F931F0E94F71A0E941D
:103850007A1A789481E0D2CF90939F0180939E0151
:10386000089590935D0280935C0208950E94231254
:10387000811103C0809157020895E0915C02F0919C
:103880005D02309729F00190F081E02D09950895AF
:1038900080E00895E0915C02F0915D02309721F0A4
:1038A0000280F381E02D09950895E0915C02F0918A
:1038B0005D02309739F022E0DC012C930480F58121
:1038C000E02D0995089520915A0230915B02281746
:1038D000390771F090935B0280935A02E0915C0289
:1038E000F0915D02309721F00680F781E02D099577
:1038F000089520915802309159022817390771F024
:103900009093590280935802E0915C02F0915D021D
:10391000309721F00084F185E02D099508959C01F0
:103920002E5F3F4FAC01485F5F4F80E024173507A3
:1039300009F40895F90191919F019923B9F38F5FDB
:10394000F5CF662349F0FC0132960896219126179F
:1039500029F0E817F907D1F780E0089581E008958C
:103960009C01FC0132969FEF80E04191461751F097
:103970009F3F19F4411101C0982F8F5F8630A9F73E
:103980009F3F09F40895290F311D97FD3A95F901DC
:1039900062830895FC01329608962191261303C094
:1039A000DF0111971C92E817F907B9F708950E94F3
:1039B000B01C08950E94CA1C0895029626E0FC01DE
:1039C00011922A95E9F7089546E050E00E944A25B1
:1039D00021E0892B09F420E0822F089508950E94A8
:1039E000EE1C0895811106C081E080935E020E9462
:1039F000EF1C089582E0F9CF83E080935E020E947D
:103A0000EF1C08950E94F21C089581E080935E02ED
:103A10000E94EF1C08950E94051D089508950895C1
:103A20000E940F1D0895089508950E940E1D089587
:103A3000CF930E94131D0E94A7110E94141DC0E085
:103A40008C2F0E947910811105C0CF5FC830C1F75B
:103A5000CF91089581E0FCCF85B7806885BF85B799
:103A6000806885BF08951F921FB61F9211248F93FF
:103A70009F93AF93BF9380915F02811113C0809198
:103A8000850290918602A0918702B09188024196AA
:103A9000A11DB11D8093850290938602A093870299
:103AA000B0938802BF91AF919F918F911F901FBEDD
:103AB0001F90189580918D02843031F10E9453033C
:103AC00010925F0288E190E020E40FB6F894A89588
:103AD000809360000FBE2093600083B7817F846075
:103AE00083BF83B7816083BF7894889583B78E7FC7
:103AF00083BF0FB6F894A895809160008861809389
:103B00006000109260000FBE08950E943B070E9463
:103B10005803089582E084BD93E095BD9AEF97BD68
:103B200080936E0008952FB7F8948091850290914C
:103B30008602A0918702B09188022FBF08952FB707
:103B4000F89460918502709186028091870290912D
:103B500088022FBF08959C014FB7F8948091850289
:103B600090918602A0918702B09188024FBF821B7C
:103B7000930B0895CF92DF92EF92FF922FB7F894B4
:103B8000C0908502D0908602E0908702F090880273
:103B90002FBFA7019601261B370B480B590BCA01F3
:103BA000B901FF90EF90DF90CF90089578941F9225
:103BB0001FB61F9211248F939F93AF93BF93809151
:103BC000850290918602A0918702B09188020196A9
:103BD000A11DB11D8093850290938602A093870258
:103BE000B0938802BF91AF919F918F911F901FBE9C
:103BF0001F90189587E797E7909301088093000836
:103C000088E19AE00FB6F894A895809360000FBE03
:103C100090936000FFCF88E19AE00FB6F894A895E2
:103C2000809360000FBE90936000FFCF80916B0285
:103C3000089508959C0182E08093E9009FEF8091B0
:103C4000E800915085FD06C085ED8A95F1F70000EA
:103C50009111F5CF8091E80085FF0CC050E040E065
:103C600066E070E0C9010E944C208091E8008E77E8
:103C70008093E8000895CF93DF93EC0181E0809377
:103C8000E9008FEF9091E800815095FD06C095ED19
:103C90009A95F1F700008111F5CF8091E80085FF3A
:103CA00014C050E040E068E070E0CE010E944C207B
:103CB0008091E8008E778093E80088E0FE01A3E61B
:103CC000B2E001900D928A95E1F7DF91CF910895CE
:103CD00080936002709362026093610280918D0212
:103CE000843001F582E08093E9008FEF9091E80045
:103CF000815095FD06C095ED9A95F1F70000811170
:103D0000F5CF8091E80085FF0DC050E040E063E012
:103D100070E080E692E00E944C208091E8008E776F
:103D20008093E8000895BC0184E00E94681E089515
:103D3000BC0183E00E94681E089580918C0281116D
:103D400009C00E94DC210E9439228091E200846037
:103D50008093E200089510928C0208950E94051D40
:103D600008956091890281E0611101C080E00E94A4
:103D7000FC1C089590918D0281E0943009F080E060
:103D8000609189020E94021D089542E061EC81E089
:103D90000E94582142E261EC82E00E9458219091F9
:103DA0008D0281E0943009F080E0609189020E94E8
:103DB000F21C089580918F02833009F461C030F4C1
:103DC0008130D1F1823009F49EC008958A3009F41F
:103DD0008AC08B3009F46FC0893009F050C08091DF
:103DE0008E02813209F04BC0809192029091930231
:103DF000029708F044C08091E800877F8093E80034
:103E00008091E80082FF37C09091F3008091F2002A
:103E1000029731F48091F100813011F0863021F465
:103E20008091F10080936B028091E8008B77809302
:103E3000E8000E948C2123C080918E02813AF9F41F
:103E40008091E800877F8093E800809192029091B2
:103E50009302892B61F468E083E692E070E00E94AF
:103E60009B208091E8008B778093E800089560E0C4
:103E700090E080E0F3CF80918D028111C1CF089551
